:10437F000000B30101010200000301FA0400FA0575
:10438F0000020A0A5A0B000F0C00FA0D00030E0070
:10439F00030F0132100096120132130AFA140102B0
:1043AF0015010217010A18010A1905321A010A1B11
:1043BF00010A1C053223011E2400642A00FA2B0077
:1043CF00FA2C50782D003C2E00462F001E30006432
:1043DF003250783300003432FA35016436016437D5
:1043EF000150380A643C00643E003C3FFFFF40FF31
:1043FF00FF411450420A5A430AC844053245007817
:10440F004600FA47FFFF4802034C00FA4EFFFF50E9
:10441F000404510596520A32530B28540A9656013A
:10442F0002570546580002590A465A32FA5B010AEA
:10443F005C0A325E000A5F00FE61FFFF64FFFF67E8
:10444F0001036A0A3C6B00006C32967801327901E5
:10445F0032FAFAFA0000B30101010200000301FA77
:10446F000400FA0500020A0A5A0B000F0C00FA0D9D
:10447F0000030E00030F0132100096120132130ACF
:10448F00FA14010215010217010A18010A1905325F
:10449F001A010A1B010A1C053223011E2400642A7B
:1044AF0000FA2B00FA2C50782D003C2E00462F00DE
:1044BF001E3000643250783300003432FA35016414
:1044CF00360164370150380A643C00643E003C3FBB
:1044DF00FFFF40FFFF411450420A5A430AC84405E8
:1044EF00324500784600FA47FFFF4802024C00FAB7
:1044FF004EFFFF500404510596520A32530B2854B5
:10450F000A96560101570546580001590A465A3274
:10451F00FA5B010A5C0A325E000A5F00FE61FFFF70
:10452F0064FFFF6701036A0A3C6B00006C329678E8
:10453F000132790132FAFAFA0065006F00790083CF
:10454F00008D009700A100AC00B600C000CA00D4D7
:10455F0000DE00E800F2005B0063006A0072007A80
:10456F00008200890091009900A100A800B000B856
:10457F0000BF00C700CF00D600DF00E600EE00F658
:10458F0000400046004C00520059005F0065006B70
:10459F0000710077007D00830089008F0095009CDB
:1045AF0000A200A800AE00B400BA00C000C600CC44
:0C45BF0000D200D900DF00E500EB00F1A5
:10009E00AE32AF3374B48E048F05FF1200858C34EC
:1000AE008D35AE32AF3374B48E048F05FF12484EC9
:1000BE008C328D33E5334532601374B4C39533FF00
:1000CE00E49532FE8E328F33783412489A229000A5
:1000DE0073E0B40104C20D8002D20D900074E0B43E
:1000EE000104C20E8002D20E9000B1E075F0DCA4C5
:1000FE00FFAEF0740A8E048F05FF120085900799EB
:10010E00ECF0A3EDF0A208401674038C068D0712D6
:10011E0048337401124825900797EEF0A3EFF07E56
:10012E00017F0090006FE01248339000B2E08E0421
:10013E008F05FF120085740AFF1200858D3890001E
:10014E00BBE075F0DCA4FFAEF0740A8E048F05FFE1
:10015E0012008590079DECF0A3EDF09000BDE060DD
:10016E00139000BDE0F5F0741684FF7E00EF90074B
:10017E00A5F0800674649007A5F090009CE0B40B87
:10018E000874E390005EF0804990009CE0B4191270
:10019E009000B2E0904532124816E49390005EF063
:1001AE00803090009CE0B41E129000B2E09045505A
:1001BE00124816E49390005EF0801790009CE0B415
:1001CE0028109000B2E090457A124816E493900001
:1001DE005EF090003AE0C39405502274019000B591
:1001EE00F09000B7E0B4020674019000B7F09000F2
:1001FE00A7E0D39402400674029000A7F09000CFBF
:10020E00E0B40117900024740FF0A374FFF0900077
:10021E0026E4F0A3F074029000CFF09000CFE0B48B
:10022E000341900026E0FEA3E0FF900024E0FCA333
:10023E00E0FD12489274101248337408124825EFEC
:10024E0090005BF0EF700674FF90005BF07400900E
:10025E0000CFF0900025E090005CF0900024E0903C
:10026E00005DF090002C7401F0740290002DF022CD
:10027E00C293C294C291C292C287C290E5B554EFA6
:10028E00F5B5E5B554DFF5B5C296C295C2A0C297D5
:10029E00C2A2C2A1E5B5547FF5B5E5B554BFF5B51B
:1002AE00E5B554FBF5B5C20F7536469000A9E07062
:1002BE0005754802800375480390000C74FFF0A387
:1002CE0074DCF090008AE0900012F8E4F0E8A3F0FD
:1002DE00C214C21674C8900028F074C890002AF098
:1002EE00752500752400C208756B00E54AB4090334
:1002FE00754A00753B0090001AE4F0A3F0754B1E92
:10030E00752700752600C212C213900799E0FEA34E
:10031E00E0FF74031248337401124825900797EEDC
:10032E00F0A3EFF0C203900010E4F0A3F0C21D2280
:10033E00053C2285A74E75A7109000A7E0B4031EBA
:10034E00A2D8B34002C293A2D9B34002C294A2DA99
:10035E00B34002C291A2DBB34002C2928012A2D875
:10036E00B34004C293C291A2D9B34004C294C292C4
:10037E00A2DCB34002C287A2DDB34002C29075D8A0
:10038E0040854EA722900047E4936406600280FEEB
:10039E0074C890079FF8E4F0E8A3F075B500758473
:1003AE000175A70075FF8075EF0690002EE4F075BD
:1003BE00C91075A70F75A1C775A70075D90075CEA1
:1003CE000C75A70F75F1FE75F2FF75F30775F478CE
:1003DE0075A4BA75A5FF75A60775AE0075AFFF7546
:1003EE00D48175D5FF75D6FF75D7FF75A70075A299
:1003FE000175A14775F80975D80075D90475A71050
:10040E0075D80075D90475DA0975DB0975DC0975BF
:10041E00DD0975DE0975DF0975D84075A70075E62B
:10042E000075E71075BC0175BE0475BD6C75BE0711
:10043E0075BDA075BE0875BD0175BC0075BB187580
:10044E00BC2075BA0875E88075D11375B50075A70F
:10045E000F75E10575E20075C740C293C294C29153
:10046E00C292C287C290E5B554EFF5B5E5B554DF3B
:10047E00F5B5C296C295C2A0C297C2A2C2A1E5B5F9
:10048E00547FF5B5E5B554BFF5B5E5B554FBF5B5F7
:10049E00759700759780740A1200757597C0E59769
:1004AE005420700280F8758F0275A700D2AF759830
:1004BE000075A90C75A70F75AB4375ADFB75AC1E1A
:1004CE0075A71075C91875CA0075CB0075C8047567
:1004DE00A700758912758E04758C00758A00C2A9E5
:1004EE00D28C758D00758B00D2ABD28E75D94475BA
:1004FE003100753000752D00752C00754500754660
:10050E0000C2997509C87508001227D575B5007413
:10051E006390079FF8E4F0E8A3F0122A617509646E
:10052E007508001227D5C21C900049E0B40108A23C
:10053E00B54002D21C802E900049E0B4021175A77E
:10054E000F75F30F75A700A2A34002D21C80169060
:10055E000049E0B4030F75A70F75F31775A700A236
:10056E00A44002D21CA21CB3500302065A74089077
:10057E00079FF8E4F0E8A3F01229307509647508B6
:10058E00001227D5740990079FF8E4F0E8A3F01243
:10059E0029307509647508001227D5740A90079FD3
:1005AE00F8E4F0E8A3F0122930750964750800121A
:1005BE0027D5740B90079FF8E4F0E8A3F0122930CA
:1005CE007509647508001227D5740C90079FF8E41E
:1005DE00F0E8A3F01229307509647508001227D5CA
:1005EE00740D90079FF8E4F0E8A3F0122930750916
:1005FE00647508001227D5740E90079FF8E4F0E892
:10060E00A3F01229307509647508001227D57402FB
:10061E009000A8F0900049E090006CF0900049E046
:10062E00B401087400900074F0801C900049E0B48E
:10063E00020874009000B7F0800D900049E0B403FA
:10064E000674009000C4F0D21902073390079FE49D
:10065E00F0A304F01229307509647508001227D52D
:10066E00740290079FF8E4F0E8A3F01229307509A0
:10067E00647508001227D5740390079FF8E4F0E81C
:10068E00A3F01229307509647508001227D5740479
:10069E0090079FF8E4F0E8A3F0122930750964750D
:1006AE0008001227D5740590079FF8E4F0E8A3F030
:1006BE001229307509647508001227D57406900743
:1006CE009FF8E4F0E8A3F01229307509647508006C
:1006DE001227D5740790079FF8E4F0E8A3F01229CB
:1006EE00307509647508001227D574019000A8F0C2
:1006FE00900049E090006CF0900049E0B40108745D
:10070E0000900074F0801C900049E0B40208740060
:10071E009000B7F0800D900049E0B403067400908D
:10072E0000C4F0C219122BD59000B2E07006740A04
:10073E009000B2F090005EE0700674E390005EF000
:10074E001200DCE5B54401F5B57406900038F0747E
:10075E0001900039F0740390003BF0740490003C5B
:10076E00F0743090003DF0740590003EF090003A29
:10077E00E0B40406740490003EF0740390003FF061
:10078E007400900044F07400900045F074019000E5
:10079E0046F07400900047F074FF900048F0744DDE
:1007AE00900136F07469900137F07474900138F04E
:1007BE007473900139F0747590013AF0746290017F
:1007CE003BF0746990013CF0747390013DF07468D5
:1007DE0090013EF0746990013FF07420900140F05A
:1007EE007434900141F07443900142F07479900199
:1007FE0043F09000CEE090005BF0900085E090001A
:10080E005CF0900086E090005DF0C214C21674C8D1
:10081E00900028F074C890002AF0C212C213A2B63B
:10082E00B3920BA2B3B3920CC209C20A752500751E
:10083E002400753646754B1E900057E4F075261948
:10084E0075276490000C74FFF0A374DCF0C20F7572
:10085E004A00C208752900752800900010E4F0A324
:10086E00F0743A90075FF074FD900760F0756C00BD
:10087E00900058E4F0752B00752A00900014E4F0F7
:10088E00A3F090008AE0900012F8E4F0E8A3F09054
:10089E00006BE075F032A4FFAEF0900022EEF0A3F4
:1008AE00EFF0900799E0FEA3E0FF74031248337453
:1008BE0001124825900797EEF0A3EFF075490174E9
:1008CE00FA900034F0C21D756B00753B00C210C269
:1008DE0011C21EC203754C00C204D205C206D20755
:1008EE00C21AC21B74FE90002FF074FE900030F0FE
:1008FE00753700754300753900753D32753E0075CC
:10090E003F00743C900032F0743C900033F0754020
:10091E000075410075420090001AE4F0A3F0754492
:10092E0000D2B2D2A4D2B0D2B1D2A3D2A7D2A6D282
:10093E00A5D2B790006BE0D394FA400674FA9000FB
:10094E006BF07E017F0090005DE012483390005CFA
:10095E00E02FFF50010E900024EEF0A3EFF0EFD346
:10096E0094FFEE940F4007900024E4F0A3F0900063
:10097E005BE0700674FF90005BF09000A8E0D394EB
:10098E0002400674019000A8F09000A9E070057571
:10099E00480280037548039000AAE0D394014006F4
:1009AE0074009000AAF09000B0E0C3940A50067450
:1009BE000A9000B0F09000BAE0700674019000BA90
:1009CE00F09000BAE0B4FF0674FE9000BAF090000A
:1009DE00C1E0D394FE400674FE9000C1F074019005
:1009EE0000C7F074019000C8F074009000CAF07453
:1009FE00009000CFF0D29CD2EC75CF01A298B350EC
:100A0E0003020DF7C298E54664046006E59964FF9B
:100A1E006002801EE546600874E62546900034F0BC
:100A2E00754600E545600874F02545900034F07574
:100A3E004500E5466003020AE2754600E599B4FFFB
:100A4E0003754501E599B4FE03754502E599B4FDBC
:100A5E0003754503E599B4FC03754504E599B4FAAD
:100A6E0003754505E599B4FB03754601E599B4F99F
:100A7E0003754604E599D394E54007E599C394F0D0
:100A8E00400280168599477546027E017F00E54734
:100A9E00C394E61248338E2E8F2F753100753000B9
:100AAE00E599D394C74007E599C394E64002801FA9
:100ABE0085994775460374E5C39547F52F752E0046
:100ACE00AE2EAF2F9045CB1200647830124878D2FC
:100ADE0099020DF7E546B401028003020BBEE53123
:100AEE004530700312027EAE30AF3190005F124877
:100AFE005AE599F0783012489AAE30AF31EFB40122
:100B0E0006EEB407028003020BBE90075FE0B43C12
:100B1E00028003020BA8C29C1200DC90005BE090E6
:100B2E0000CEF090005CE0900085F090005DE090CB
:100B3E000086F0A2194031754F01E54FD39407504E
:100B4E0025E54F90079FF8E4F0E8A3F074AA900013
:100B5E002EF01228017509647508001227D5784FFA
:100B6E00740126F650D4802F754F08E54FD3940E9E
:100B7E005025E54F90079FF8E4F0E8A3F074AA9093
:100B8E00002EF01228017509647508001227D57819
:100B9E004F740126F650D4122BD574C890079FF8C7
:100BAE00E4F0E8A3F0D29C7546007545007599FBFC
:100BBE00E546B402028003020C52E5314530700660
:100BCE0085992D752C00AE30AF3174016F4E701BB0
:100BDE00AC2CAD2DAA2EAB2FED2BFBEC3AFA8A06E0
:100BEE008B0790005F12485AE599F0783012489AB8
:100BFE00AE30AF3174026F4E704AAC2CAD2D740D09
:100C0E006D4C7027746390079FF8E4F0E8A3F074BE
:100C1E00AB90002EF090006CE0900049F0122B3A51
:100C2E0074C890079FF8E4F0E8A3F0AE2CAF2D74D3
:100C3E00566F4E700312027E1200DC854799754680
:100C4E0000754500E546B4033FAE30AF3190005F0E
:100C5E0012485AE599F0783012489AAE30AF31AC5E
:100C6E002EAD2F8F028E038C068D07904607120035
:100C7E0064E493F9740193FEEAD39EEB99400985DF
:100C8E004799754600754500E546B4040280030297
:100C9E000DF7E5314530700312027EAE30AF319064
:100CAE00005F12485AE599F0783012489AAE30AF8C
:100CBE0031EFB40006EEB401028003020DF790008E
:100CCE0042E075F002A4FDACF08D4FED90005F1286
:100CDE00486FEDFAE0FBEA90006212486FEBFAE023
:100CEE00FBEA2BFA900042E0B502028003020DE906
:100CFE000DED90005F12486FE54FFDE0FAED9000AC
:100D0E006312486FEAFDE0FAEDC39AFD900042E0EF
:100D1E00B505028003020DE9E54F90006112486FA0
:100D2E00E54FFDE0FAED90006412486FEAFDE0FA3F
:100D3E00ED2AFD900042E0B505028003020DE9E5C3
:100D4E004F90006512486FFDE0FAED900042E0F41E
:100D5E00042A900049F0E54F90006612486FFDE0BE
:100D6E00FAED900042E0F4042A90004AF0E54F902C
:100D7E00006712486FFDE0FAED900042E0F4042A9D
:100D8E0090004BF0E54F90006812486FFDE0FAEDD1
:100D9E00900042E0F4042A90079FF8E4F0E8A3F0F4
:100DAE0074AB90002EF0122B3A7509647508001280
:100DBE0027D590079F124841122B3A750964750882
:100DCE00001227D590079F124841122B3A7599F9B8
:100DDE007509647508001227D580FE7599FF75098F
:100DEE00647508001227D580FEE5456006A299B30A
:100DFE00B34003020F75C299E545B4011FAE30AF83
:100E0E003190003812485AE0F599783012489AAE6F
:100E1E0030AF3174116F4E7003754500E545B40265
:100E2E0003854999E545B4031DAE30AF3190005F9F
:100E3E0012485AE0F599EFB40107EEB40703754571
:100E4E0000783012489AE545B404028003020F3749
:100E5E00E53145307003852599AE30AF3174016FA1
:100E6E004E7003853799AE30AF3174026F4E7003FA
:100E7E00853999AE30AF3174036F4E7003853D994D
:100E8E00AE30AF3174046F4E7003853F99AE30AF04
:100E9E003174056F4E7003854099AE30AF317406D4
:100EAE006F4E7003854199AE30AF3174076F4E703F
:100EBE0003854299AE30AF3174086F4E70069000C4
:100ECE001BE0F599AE30AF3174096F4E700690008D
:100EDE0034E0F599AE30AF31740A6F4E700385432E
:100EEE0099AE30AF31740B6F4E7003853E99AE30B4
:100EFE00AF31740C6F4E7003854499AE30AF3174C0
:100F0E000D6F4E7005900034E4F0AE30AF31740DBD
:100F1E006F4E70037599FC783012489AAE30AF312F
:100F2E00740E6F4E7003754500E545B4053990009B
:100F3E003AE0D394044010AE30AF3190437F124864
:100F4E005AE493F599800EAE30AF31904463124857
:100F5E005AE493F599AE30AF3174E36F4E7003756A
:100F6E004500783012489AE54664016005E546B4BE
:100F7E000403020A07C28E7E087F00E53C12483346
:100F8E00E58D75F008A4FDACF0EF2DFDEE3CFCE513
:100F9E008B75F02084FF7E00ED2FFFEC3EFE8E263B
:100FAE008F27D28E90008CE0605690001C12484124
:100FBE0090001CE0FCA3E0FD90001EE0FAA3E0FB15
:100FCE00EDB5033CECB50238B218A208B34013A23B
:100FDE0018B34008E5B54404F5B58006E5B554FBF5
:100FEE00F5B590001EE0FEA3E0FF900020E0FCA30C
:100FFE00E0FDEF2DFDEE3CFC90001EECF0A3EDF0BD
:10100E00900099E06009900099E0C394034002803B
:10101E007A1240D5A208B35009900057E0C3942825
:10102E0040028006900083E0F56AE56A75F005A43B
:10103E00FFAEF09007A1EEF0A3EFF0900070E0C3CA
:10104E0095394007E537C3953850079007A1E4F06E
:10105E00A3F0AE57AF589007A1E0FCA3E0FDEFD38D
:10106E009DEE9C4004C2A1800B900057E0C3943CBF
:10107E005002D2A1900099E0B402099000A7E0C3FB
:10108E00940340028005A2A1B392A2900099E0B40D
:10109E00031C1241D1AE57AF589007A1E0FCA3E05C
:1010AE00FDEFD39DEE9C4004D2A18002C2A1A2B35B
:1010BE00300C01B34029A2B3300C01B34021A2B3CE
:1010CE00300E01B34005A20EB3920CA20EB330B394
:1010DE0001B3400BA2B6B34002D21AA20E920CA2DA
:1010EE00B6300B01B3500302151FA2B6300B01B37D
:1010FE00500302151FA2B6300D01B3500302145156
:10110E0075490090008CE07013A20DB34008E5B550
:10111E0054FBF5B58006E5B54404F5B50536A2B326
:10112E00300E01B350030211BDE548B40330E5366D
:10113E00B40305754801801FA21DB3401AE536C3DE
:10114E00940350069000347401F0E536D3940340B6
:10115E00067402900034F0753601D21D8044E548C5
:10116E00B40206754801753603E536B403057536C7
:10117E0001802F900034E0701AE536C394035006B8
:10118E009000347401F0E536D39403400674029057
:10119E000034F09000A9E0B4020512027E800375BF
:1011AE003601A21AB34004D21B8002C21BC21AE53A
:1011BE0048C394035006E536640360028005753615
:1011CE0001C21BE536B4024990008CE060439000EA
:1011DE001CE0FEA3E0FF90008CE08E048F05FF1252
:1011EE00008574018C068D07124825900020EEF0C4
:1011FE00A3EFF0900020E0F8A3E090001EC8F0A34B
:10120E00C8F090001CE4F0A3F0C218E5B554FBF54D
:10121E00B5AE2AAF2BAC26AD27EF2DFDEE3CFC8CE8
:10122E002A8D2BAE26AF27EFD39DEE9C401190005A
:10123E0014E0FAA3E0FBEBC394E8EA9403400280C7
:10124E000690001412484190000CE526F0A3E52705
:10125E00F090000EE526F0A3E527F0AE26AF27743A
:10126E00128E048F05FF1200858C288D29C28E7573
:10127E008D00758B00753C00752701752600D28E8A
:10128E0090000CE0FEA3E0FFEF4E600B7C827D4CE5
:10129E001247358E248F25AE24AF257428BE000349
:1012AE009F5010E53B2FFF50010E74011248258E02
:1012BE00248F2585253B75CD0075CC00753C00909F
:1012CE0000B0E0A824B8000DD395254008E5259080
:1012DE000031F080099000B0E014900031F0E54844
:1012EE006006752500752400123E17E54AB4090301
:1012FE00754A00A21050030213DE900065E0B4019F
:10130E005AE53F75F00584FF7E0090055F12485A3E
:10131E00E0F533753200AE32AF33900063E0124821
:10132E003374648E048F05FF12008574C18C068D94
:10133E00071248338E348F35900012E0FEA3E0FF83
:10134E00AC32AD3312000374648E048F05FF1200AD
:10135E0085900012ECF0A3EDF0800F900063E07525
:10136E00F0C1A4FFAEF08E348F35E539C394CC5066
:10137E005D75A71085F94F85FA507E017F00E55007
:10138E00124833E54F2FFF50010E8E328F33AC349F
:10139E00AD35EF2DFDEE3CFC8C348D35D293D294D1
:1013AE00E535F5FBE534F5FCE535F5E9E534F5EA2B
:1013BE009000A7E0B40314D291D292E535F5EBE597
:1013CE0034F5ECE535F5EDE534F5EE75A700D21004
:1013DE00E548B4010F754B019000377401F0E5B587
:1013EE004401F5B5E54870569000ACE0600D9000F4
:1013FE00B3E0A824B800069525400280239000ACE7
:10140E00E0B40208754B03754400800CC2007544AD
:10141E000090001AE4F0A3F07409900034F0801EDE
:10142E00E536B4010B754B019000377401F0800E58
:10143E00E536B40209754B017402900037F0A20D27
:10144E00B3920BA20DB330B601B3500302151F7544
:10145E004901A20D920BE536D394484012D20FE506
:10146E0036D3944C40097403900034F07536469090
:10147E0000B4E0B40107E542C394144002800312A5
:10148E00027E7428900057F0A204300501B3501765
:10149E00A204B34008E5B54408F5B58006E5B55499
:1014AE00F7F5B5A2049205A206300701B35017A2B4
:1014BE0006B34008E5B54402F5B58006E5B554FD22
:1014CE00F5B5A2069207E542C394415009740E90F9
:1014DE000034F012027E90003EE0FE90003AE004EE
:1014EE00C39E400990003AE0D39406400974FB90E5
:1014FE000034F012027E900043E06015900043E04D
:10150E00FE90003DE06E600974FE900034F0120211
:10151E007EA212B3B35006E536640260030215FBD9
:10152E00A202B35006A200B3B340030215F775A78B
:10153E001085F94F85FA507E017F00E55012483331
:10154E00E54F2FFF50010E8E328F33900018E0FCC6
:10155E00A3E0FDEF2DFDEE3CFC8C348D359000A705
:10156E00E0B4034EA208B34028A21BB3400CE535ED
:10157E00F5FBE534F5FCD293800AE535F5EBE53461
:10158E00F5ECD291A203B34004D2A08002C2A08097
:10159E001FE535F5FBE534F5FCE535F5EBE534F502
:1015AE00ECD293D291A203B34004D2A08002C2A087
:1015BE008011E535F5FBE534F5FCD293A203B3407B
:1015CE0002D2919000C5E0B4021CAE32AF33AC55DE
:1015DE00AD56EF2DFDEE3CFC8C348D35E535F5FD2D
:1015EE00E534F5FED28775A700C212D213A213B34B
:1015FE00B35006E536640160030216D7A202B3505B
:10160E0006A200B3B340030216D375A71085F94F97
:10161E0085FA507E017F00E550124833E54F2FFFCB
:10162E0050010E8E328F33900018E0FCA3E0FDEFD8
:10163E002DFDEE3CFC8C348D359000A7E0B4034EAE
:10164E00A208B34028A21BB3400CE535F5E9E534FA
:10165E00F5EAD294800AE535F5EDE534F5EED29251
:10166E00A203B34004D2A08002C2A0801FE535F5CC
:10167E00E9E534F5EAE535F5EDE534F5EED294D24B
:10168E0092A203B34004D2A08002C2A08011E5351D
:10169E00F5E9E534F5EAD294A203B34002D2929072
:1016AE0000C5E0B4021CAE32AF33AC55AD56EF2DD3
:1016BE00FDEE3CFC8C348D35E535F5CEE534F5CFBD
:1016CE00D29075A700D212C213E54BB4081612378A
:1016DE0046A212B35005A213B340028004D212D216
:1016EE0013754B1EE54BB407061234FE754B08E519
:1016FE004BB4063D900012E0FEA3E0FFEF4E6006F5
:10170E00A208B3B340028023AE51AF52900012E054
:10171E00FCA3E0FDEF2DFDEE3CFC8C518D52E53629
:10172E00D3940150069000121200391232D0754B2C
:10173E0007E54BB40506123130754B06E54BB40484
:10174E003290009AE09027B7F8282873122DC480A3
:10175E0012122DC4800D122F7280081230248003B5
:03176E0012302412
:0F27B70002175A02175F02176402176902176EA2
:1017710090007CE06005123F008002C204754B05B9
:10178100E54BB40302800302186B90007FE0600513
:10179100123FF08002C20690009AE0D39402403FCB
:1017A10090006EE02403A824B80004952550099008
:1017B1000070E0D3953950028008D202740890007D
:1017C10034F090006EE0A824B80005D39525500BA5
:1017D100900070E02403C395395002C20280399011
:1017E100006EE02403A824B8000495255007E537CE
:1017F100C3953840028008D2027408900034F090FA
:10180100006EE0A824B80005D395255009E53824D9
:101811000FC395375002C2029000B4E07007E54251
:10182100C3941440028002D202A2024005754B0407
:10183100800A754B1E90001AE4F0A3F0A208B34091
:1018410029E53F75F00584FF7E0090055F12485A37
:10185100E0C394695005123E4C800F900799E0F85F
:10186100A3E0900797C8F0A3C8F0E54BB40A028043
:101871000302193B900029E0C394465008C29674B4
:1018810046900029F085593375320090002CE0F51F
:101891004F12009EE535900029F0900006E532F0E8
:1018A100A3E533F0C215900060E0FE900029E0C38B
:1018B1009E5012900060E0FE900029E0F4042E900A
:1018C1000029F08012900060E02402FE900029E0DF
:1018D100F4042E900029F090079BE0F532A3E0F587
:1018E1003390002CE0F54F12009EE535900028F072
:1018F100900000E532F0A3E533F0C214900060E0FF
:10190100FE900028E0C39E5012900060E0FE90001F
:1019110028E0F4042E900028F08012900060E0246A
:1019210002FE900028E0F4042E900028F0E548B46F
:101931000105754B0B8003754B03900028E0B5360C
:101941000280030219D3A214406B900000E0FEA3B1
:10195100E0FFEF4E605DAC24AD25740ABC0033D3CB
:101961009D402FAA28AB2974058A048B05FF12001C
:10197100858D068C07900000E0FCA3E0FDCFCECF63
:101981001200037401124825900000EEF0A3EFF05D
:101991008021AE28AF29900000E0FCA3E0FD1200F9
:1019A10003740A8E048F05FF120085900000ECF08D
:1019B100A3EDF0D214AE26AF27900000E0FCA3E027
:1019C100FDEFC39DEE9C400AD296C21474C89000EC
:1019D10028F0A214B3B35007900028E0B536028076
:1019E1000AD29674C8900028F0C214900029E0B57C
:1019F10036028003021A84A215406B900006E0FEB5
:101A0100A3E0FFEF4E605DAC24AD25740ABC00334A
:101A1100D39D402FAA28AB2974058A048B05FF1298
:101A210000858D068C07900006E0FCA3E0FDCFCE7B
:101A3100CF1200037401124825900006EEF0A3EFC7
:101A4100F08021AE28AF29900006E0FCA3E0FD1252
:101A51000003740A8E048F05FF120085900006ECC6
:101A6100F0A3EDF0D215AE26AF27900006E0FCA35F
:101A7100E0FDEFC39DEE9C400AC29674469000299A
:101A8100F0C215A215B3B35007900029E0B5360294
:101A9100800AC2967446900029F0C215E54BB40B3A
:101AA100028003021B8690002BE0C39446501390E2
:101AB10000B5E0B40104C2968002C295744690005C
:101AC1002BF085593375320090002DE0F54F12004F
:101AD1009EE53590002BF0900008E532F0A3E53348
:101AE100F0C217900060E004FE90002BE0C39E500E
:101AF10013900060E004FE90002BE0F4042E9000AF
:101B01002BF08012900060E02403FE90002BE0F4A3
:101B1100042E90002BF090079BE0F532A3E0F53303
:101B210090002DE0F54F12009EE53590002AF090CF
:101B31000002E532F0A3E533F0C216900060E00444
:101B4100FE90002AE0C39E5013900060E004FE90D6
:101B5100002AE0F4042E90002AF08012900060E048
:101B61002403FE90002AE0F4042E90002AF0E548B8
:101B7100B4010F75480074C8900028F074C8900033
:101B81002AF0754B0390002AE0B536028003021C4F
:101B910029A216406B900002E0FEA3E0FFEF4E6029
:101BA1005DAC24AD25740ABC0033D39D402FAA2817
:101BB100AB2974058A048B05FF1200858D068C07FD
:101BC100900002E0FCA3E0FDCFCECF120003740130
:101BD100124825900002EEF0A3EFF08021AE28AF6D
:101BE10029900002E0FCA3E0FD120003740A8E04B8
:101BF1008F05FF120085900002ECF0A3EDF0D216E4
:101C0100AE26AF27900002E0FCA3E0FDEFC39DEEFE
:101C11009C40159000B5E0B40104D2968002D295A3
:101C2100C21674C890002AF0A216B3B350079000F0
:101C31002AE0B5360280159000B5E0B40104D296D1
:101C41008002D29574C890002AF0C21690002BE051
:101C5100B536028003021CF0A217406B900008E029
:101C6100FEA3E0FFEF4E605DAC24AD25740ABC001D
:101C710033D39D402FAA28AB2974058A048B05FF15
:101C81001200858D068C07900008E0FCA3E0FDCFD3
:101C9100CECF1200037401124825900008EEF0A384
:101CA100EFF08021AE28AF29900008E0FCA3E0FD11
:101CB100120003740A8E048F05FF1200859000083C
:101CC100ECF0A3EDF0D217AE26AF27900008E0FCB0
:101CD100A3E0FDEFC39DEE9C40159000B5E0B4017B
:101CE10004C2968002C295744690002BF0C217A2DE
:101CF10017B3B3500790002BE0B536028015900062
:101D0100B5E0B40104C2968002C295744690002BDE
:101D1100F0C217E54BB402028003021DC2123BAFB1
:101D2100123CC690005FE02544F559900797E0FE0C
:101D3100A3E0FF740A12483390000EE0FCA3E0FD1B
:101D410074098F02FF1200858D078C038E048A05AA
:101D51008B0612473590079BEEF0A3EFF09000B58C
:101D6100E0B401087478BE00059F4002800D7478CC
:101D710090079BF8E4F0E8A3F0801B90079BE0FE3E
:101D8100A3E0FF74F0BE00039F500B74F090079B1B
:101D9100F8E4F0E8A3F090079BE0FEA3E0FFE5592B
:101DA1002FFF50010E90079BEEF0A3EFF09000374C
:101DB100E0B40103754B0A900037E0B40203754BA0
:101DC1000BE54BB401259000CCE09027C6F82828FC
:101DD1007312394D801212394D800D1239D7800896
:081DE100123A838003123A83D9
:0F27C600021DD2021DD7021DDC021DE1021DE61D
:101DE900754B029000B7E0B402028003021F049011
:101DF900005AE0D3953E506490005AE0F404253E21
:101E0900FE9000BAE08E00F5F0E884FF7E008F4F67
:101E1900EFC39410500CEF854FF0A4FDACF08D4F3B
:101E29008003754FFF90005AE0D3954F400B900007
:101E39005AE0C3954FF54C8003754C009000D5E0EE
:101E4900D3954C40069000D5E0F54C9000D6E0C300
:101E5900954C50069000D6E0F54C807190005AE000
:101E6900C3953EFE9000BAE08E00F5F0E884FF7E4F
:101E7900008F4FEFC39410500CEF854FF0A4FDACC9
:101E8900F08D4F8003754FFF854F337532009000F9
:101E99005AE02533FFAE3250010E8E328F3374FF74
:101EA900BE0009D39F400585334C8003754CFF90D4
:101EB90000D5E0D3954C40069000D5E0F54C900054
:101EC900D6E0C3954C50069000D6E0F54CA208B375
:101ED900B350099000C2E0D3954D5002800A7407AF
:101EE900900034F0C297801375A710E5CDC3954CC7
:101EF9004004C2978002D29775A700E54AC39409A6
:101F09004003022559A2EDB35003022559C2EDE55C
:101F19004A6003021FD7900068E07003021FC67E63
:101F2900017F00E5BE124833E5BD2FFF50010E8E3B
:101F3900328F33900068E0B401187410124833905E
:101F4900005EE08E048F05FF120085ED90002FF0F2
:101F5900802CAE32AF33741012483390005EE08E9D
:101F6900048F05FF12008590002FE02DFD50010C14
:101F790074018C068D07124825EF90002FF0E54378
:101F890060089000C4E06402600280219000C6E00D
:101F9900B4011A90002FE075F0E7A4FFAEF0E54315
:101FA9008E048F05FF120085ED90002FF090009AA6
:101FB900E06401600690002FE0F537800375370073
:101FC900900064E07005754A01800375BB18E54A05
:101FD900B40102800302216F900064E070030221C2
:101FE9005E7E017F00E5BE124833E5BD2FFF50013B
:101FF9000E8E328F339000AAE0B4010F7E0F7FFF5F
:10200900AC32AD331248928E328F339000CFE0B4A8
:102019000245AE32AF33900024E0FCA3E0FDEDD3DE
:102029009FEC9E400A900024E532F0A3E533F0AE20
:1020390032AF33900026E0FCA3E0FDEFD39DEE9C88
:10204900400A900026E532F0A3E533F0AE32AF3313
:1020590074041248258F399000CFE0704CAE32AF2E
:1020690033900024E0FCA3E0FDEFD39DEE9C4009F2
:102079001248928E328F338006753300753200AE66
:1020890032AF33741012483390005BE08E048F0531
:10209900FF1200858C328D337400D39D74019C40EE
:1020A9000585333980037539FF90009AE0B4010240
:1020B900800302215CA208B3B3500E90006EE0A821
:1020C90024B80005D39525500302215690006FE0EE
:1020D90075F019A4FFAEF09000B2E08E048F05FFF1
:1020E9001200859000ABE08539F0A4FFAEF074646E
:1020F9008D028C038E048F05FF120085EA2DFDEBFE
:102109003CFC8C328D33E543600F9000C4E0B4028F
:10211900089000C6E0640160028017AE32AF3374E4
:10212900E7124833E5438E048F05FF1200858C3290
:102139008D3390002FE0A832B8000AD395334005BB
:10214900853337800690002FE0F537800690002F01
:10215900E0F5378003753900900067E07005754A2E
:1021690002800375BB19E54AB40202800302222AE0
:10217900900067E07003022219E536D39401400309
:10218900022217900022E0FEA3E0FFE53D12488AF3
:10219900900022EEF0A3EFF07E017F00E5BE124829
:1021A90033E5BD2FFF50010E8E328F339000D4E0FE
:1021B9007013740A12483374518E048F05FF12008C
:1021C900858D3D8019AE32AF33740A1248338F04BE
:1021D9008E057E017F95CDCCCD1247358F3DE53DEE
:1021E900D394644003753D64900022E0FEA3E0FFB0
:1021F900E53D2FFF50010E900022EEF0A3EFF09085
:10220900006BE0048E048F05FF1200858D3D80036D
:10221900753D329000B7E07005754A03800375BBC0
:1022290013E54AB4035E9000B7E060477E017F0082
:10223900E5BE124833E5BD2FFF50010E8E328F33B4
:1022490074041248258F3E9000B9E0853EF0A4FD44
:10225900ACF07464FF1200858D3E9000B8E0853EB5
:10226900F0A4FFAEF074FF8E048F05FF1200858D78
:102279004D8003753E00900065E07005754A048045
:102289000375BB17E54AB40402800302232B9000AF
:1022990065E0B4017C7E017F00E5BE124833E5BDEF
:1022A9002FFF50010E74041248258E328F3390008F
:1022B90032E06012900032E01490464393A832B89D
:1022C9000006953340028006900032E014F0900039
:1022D90032E0C394775013900032E0049046439360
:1022E900A832B80005D3953350028006900032E039
:1022F90004F0900032E0FE90008BE08E0088F0A49C
:10230900FFAEF074648E048F05FF1200858D3F8047
:1023190003753F00900066E07005754A05800375F6
:10232900BB16E54AB4050280030223BE900066E0AD
:10233900B4017C7E017F00E5BE124833E5BD2FFF65
:1023490050010E74041248258E328F33900033E009
:102359006012900033E0149046BC93A832B800068E
:10236900953340028006900033E014F0900033E08A
:10237900C394775013900033E0049046BC93A8327D
:10238900B80005D3953350028006900033E004F07D
:10239900900033E0FE900091E08E0088F0A4FFAE3B
:1023A900F074648E048F05FF1200858D40800375DB
:1023B900400075BB1FE54AB406337E017F00E5BEC8
:1023C900124833E5BD2FFF50010E8E328F33740949
:1023D90012483374E68E048F05FF1200858D4290F2
:1023E900006DE07005754A07800375BB15E54AB4B1
:1023F9000702800302250090006DE070030224EFBC
:102409007E017F00E5BE124833E5BD2FFF50010E66
:102419008E328F3374041248258F4190006DE0B4D9
:1024290001159000C1E08541F0A4FFAEF0740712D8
:102439004825EF9007A4F090006DE0B402159000D4
:10244900C1E08541F0A4FFAEF07407124825EF9072
:1024590007A3F090006DE0B4030280030224ED901D
:1024690000AEE0701CE541C3940A5002D201E54177
:10247900D394644002C20190008DE0900059F0802D
:102489006390008DE070349000C1E08541F0A4FFB5
:10249900AEF074FF8E048F05FF120085ED90005990
:1024A900F0AE24AF25741EBE0006D39F4002D201B0
:1024B900E539D394E54002C2018029E541C3940A74
:1024C900500DAE24AF25741EBE0004D39F50028068
:1024D90002D201E539D394E54002C20190008DE0B2
:1024E900900059F080037541009000C4E0700575B3
:1024F9004A08800375BB14E54AB408509000C4E04B
:1025090060397E017F00E5BE124833E5BD2FFF50DB
:10251900010E8E328F33EFD39421EE940E40057560
:1025290043FF8015AE32AF33741012483374E38E13
:10253900048F05FF1200858D4380037543009000C9
:1025490068E0600575BB1A800375BB18054AD2ECB3
:10255900AE26AF27EFD39400EE947D50030227B443
:10256900C20F7536469000A9E070057548028003D0
:10257900754803C293C294C291C292C287C290E5C0
:10258900B554EFF5B5E5B554DFF5B5C296C295C2B8
:10259900A0C297C2A2C2A1E5B5547FF5B5E5B5546D
:1025A900BFF5B5A21CB34008E5B54404F5B58006EE
:1025B900E5B554FBF5B5A211B3500EE539D3943303
:1025C9004007E539C394CC400302265EE5B54401D2
:1025D900F5B57428900057F0900063E075F064A495
:1025E900FFAEF08E348F357402BE000AD39F4006C9
:1025F90075350275340075A71085F94F85FA507E37
:10260900017F00E550124833E54F2FFF50010E8E30
:10261900328F33AC34AD35EF2DFDEE3CFC8C348D6F
:1026290035D293D294E535F5FBE534F5FCE535F57E
:10263900E9E534F5EA9000A7E0B40314D291D29207
:10264900E535F5EBE534F5ECE535F5EDE534F5EE95
:1026590075A700D211E539C3941A5002C21190002E
:102669000C74FFF0A374DCF090008AE0900012F87B
:10267900E4F0E8A3F0C214C21674C8900028F074FC
:10268900C890002AF0C212C213752500752400757E
:102699003B00C208756B0090001AE4F0A3F0754B7B
:1026A9001E900799E0FEA3E0FF74031248337401FA
:1026B900124825900797EEF0A3EFF090007CE060B8
:1026C90005123F008002C20490007FE06005123FBE
:1026D900F08002C206A204300501B35017A204B368
:1026E9004008E5B54408F5B58006E5B554F7F5B5F4
:1026F900A2049205A206300701B35017A206B340FF
:1027090008E5B54402F5B58006E5B554FDF5B5A271
:10271900069207C203752B00752A00900014E4F095
:10272900A3F090006BE075F032A4FFAEF0900022A8
:10273900EEF0A3EFF0900010E4F0A3F0C21D9000BA
:1027490058E0C3943C5019758D96758B00753C0FF4
:10275900E54AB40909900058E004F0754A00803B45
:10276900E54AB40903754A00752700752600758D79
:1027790000758B00753C00900057E0C3943C5008ED
:10278900900057E004F08006743C900057F09000E8
:1027990057E0B43C06E5B554FEF5B5E542C39441AE
:0E27A9005009740E900034F012027E020A07EE
:1045CB000000010001400160018001A001C001E079
:1045DB0002000300039603B603D603F404000500A0
:1045EB0005180530054805600578059005A805C038
:1045FB00060006140628063C066E068C00FF013FDB
:10460B00015F017F019F01BF01DF01FF02FF0395E6
:10461B0003B503D503F303FF04FF0517052F054768
:10462B00055F0577058F05A705BF05FF0613062751
:10463B00063B066F068B06A9DAD8D7D5D4D2D0CFD6
:10464B00CDCBC9C7C6C4C2C0BEBCBAB8B5B3B1AF77
:10465B00ADABA8A6A4A2A09D9B99969492908D8B8E
:10466B0089878482807E7C79777573716F6D6B69B6
:10467B00676563615F5D5B5957565452504F4D4BA5
:10468B004A4847454442413F3E3C3B3A3937363531
:10469B00343231302F2E2D2C2B2A29282726252555
:1046AB002423222121201F1E1E1D1C1C1B1A1A191C
:1046BB0019EEECEBEAE9E8E7E5E4E3E1E0DEDDDB6C
:1046CB00D9D8D6D4D2D0CECCCAC8C6C3C1BFBCBA37
:1046DB00B7B5B2B0ADABA8A5A3A09D9B9895929092
:1046EB008D8A8785827F7D7A7775726F6D6A686533
:1046FB0063615E5C5A575553514F4D4B4947454388
:10470B0042403E3C3B393836353332312F2E2D2B40
:10471B002A292827262524232221201F1E1D1D1C64
:0A472B001B1A1A1918181716161594
:1027D500750B00750A00AE0AAF0BAC08AD09EDC369
:1027E5009FEC9E401674FF12007575CF01780B742F
:1027F5000126F6500418E436F650DB2290002EE050
:10280500B4AA1C90075FE0B43C1590079FE0FEA3B7
:10281500E0FFEF4E6009741EBE0004D39F50030213
:10282500292F75350075340075F80990079FE0FE6E
:10283500A3E0FF74076F4E6006740E6F4E7006744A
:102845003A90075FF090079FE0FEA3E0FF7408BE93
:10285500001ED39F401A7E017F0890079FE0FCA3CE
:10286500E0FD1DBDFF011C1200038E328F33801F5A
:1028750090079FE0FEA3E0FF740812488A8F048E3C
:10288500057E017F08CDCCCD1200038E328F33AE8D
:1028950034AF35740CD39F74019E500302292AA2CC
:1028A500F9B3407EE5354534700375A382AE34AF88
:1028B5003574016F4E700375A300AE34AF357402E5
:1028C5006F4E700D9007A0E075F002A4FDACF08D81
:1028D500A3AE34AF3574036F4E700375A300AE34E9
:1028E500AF357403BE00039F5013AC32AD33ED2FEB
:1028F500FFEC3EFE90005B12485AE0F5A3AE34AF04
:1029050035EFB40B09EEB401057414120075AE343D
:10291500AF35EFB40B07EEB4010375F80D7834123B
:10292500489A02289490002EE4F0227535007534FB
:102935000075F80990079FE0FEA3E0FF7408BE004C
:102945001ED39F401A7E017F0890079FE0FCA3E0FD
:10295500FD1DBDFF011C1200038E328F33801F90B9
:10296500079FE0FEA3E0FF740812488A8F048E05D6
:102975007E017F08CDCCCD1200038E328F33AE346D
:10298500AF357411D39F74019E5003022A60A2F9DA
:10299500B35003022A5DE5354534700375A3D2AE05
:1029A50034AF3574016F4E700375A300AE34AF3587
:1029B50074026F4E700D9007A0E075F002A4FDAC97
:1029C500F08DA3AE34AF3574036F4E700375A3005D
:1029D500AE34AF3574046F4E700375A300AE34AFDB
:1029E5003574056F4E700375A300AE34AF357406AC
:1029F5006F4E700375A300AE34AF3574076F4E701C
:102A05000375A300AE34AF3574086F4E700375A31C
:102A150000AE34AF357408BE00039F5016AC32AD1E
:102A250033ED2FFFEC3EFE90005612485AE5A3F019
:102A350075A300AE34AF35EFB41009EEB4010574DB
:102A450014120075AE34AF35EFB41007EEB40103C0
:102A550075F80D783412489A022983227535007568
:102A6500340075F809AE34AF357417BE0004D39F32
:102A75005003022B39A2F9B35003022B36E5354535
:102A850034700375A3D2AE34AF3574016F4E700345
:102A950075A300AE34AF3574026F4E700D9007A06C
:102AA500E075F002A4FDACF08DA3AE34AF35740330
:102AB5006F4E700375A300AE34AF3574046F4E705E
:102AC5000375A300AE34AF3574056F4E700375A35F
:102AD50000AE34AF3574066F4E700375A300AE3487
:102AE500AF3574076F4E700375A300AE34AF357400
:102AF500086F4E700375A300AE34AF357408BE0081
:102B0500039F500C90004012485AE5A3F075A300AE
:102B1500AE34AF3574166F4E70057414120075AE71
:102B250034AF3574166F4E700375F80D783412484E
:102B35009A022A6A2290002EE0B4AB028003022B8F
:102B4500D475350075340075F809AE34AF35741297
:102B5500BE007CD39F4078A2F9B34070E53545347B
:102B6500700375A382AE34AF3574016F4E70037573
:102B7500A300AE34AF3574026F4E700D9007A0E020
:102B850075F002A4FDACF08DA3AE34AF3574036FC0
:102B95004E700375A300AE34AF357403BE00039FBA
:102BA500500990004512485AE0F5A3AE34AF35748C
:102BB500116F4E70057414120075AE34AF35741173
:102BC5006F4E700375F80D783412489A022B4F2218
:102BD500900035E4F0746490079FF8E4F0E8A3F002
:102BE500122A6174C890079FF8E4F0E8A3F09000FA
:102BF5004CE0B4371A900049E0900040F090004A4C
:102C0500E0900041F090004BE0900042F08046904B
:102C150000357401F0746590079FF8E4F0E8A3F0BF
:102C2500122A6174C890079FF8E4F0E8A3F09000B9
:102C35004CE0B4371A900049E0900040F090004A0B
:102C4500E0900041F090004BE0900042F080067467
:102C550002900035F0900036E4F0746690079FF816
:102C6500E4F0E8A3F0122A6174C890079FF8E4F035
:102C7500E8A3F090004BE0B43712900049E09000D3
:102C85003AF090004AE0900043F080769000367468
:102C950001F0746790079FF8E4F0E8A3F0122A6149
:102CA50074C890079FF8E4F0E8A3F090004BE0B4F7
:102CB5003712900049E090003AF090004AE0900009
:102CC50043F0803E7402900036F0746890079FF8D8
:102CD500E4F0E8A3F0122A6174C890079FF8E4F0C5
:102CE500E8A3F090004BE0B43712900049E0900063
:102CF5003AF090004AE0900043F08006740390009B
:102D050036F022E55C2533FFAE3250010E90005FB0
:102D150012485AE0F55DE55C2533FFAE3250010EF1
:102D25000FBF00010E90005F12485AE0F55E856402
:102D350060E55DB55E05855D5C8041E55ED3955DCD
:102D4500401DE55EC3955D855FF0A4FFAEF0E560CF
:102D55008E048F05FF120085ED255DF55C801DE570
:102D65005DC3955E855FF0A4FFAEF0E5608E048FD0
:102D750005FF120085EDF404255DF55C22E55ED3C3
:102D8500955D401DE55EC3955D855FF0A4FFAEF0E2
:102D9500E5608E048F05FF120085ED255DF55C80ED
:102DA5001DE55DC3955E855FF0A4FFAEF0E5608E21
:102DB500048F05FF120085EDF404255DF55C22E521
:102DC5003775F00484FF7E008F5CE53775F0048469
:102DD500ADF07C008D5F756404753201753300E5D7
:102DE5005CC3943F5005122D08800690019EE0F5C6
:102DF5005C855C52755100900031E075F020A4FFB0
:102E0500AEF09000B0E08E048F05FF1200858D5C5A
:102E1500900098E0D395375003022ECA9000BCE08D
:102E2500D395374010ED90019F12486FE0F554752A
:102E35005300022EC7900087E0D395374043E55CE9
:102E450090019F12486FE0F55DE55C9001BF124867
:102E55006FE0F55E9000BCE0F4042537F55F900067
:102E650087E0FE9000BCE0F4042EF560E55DB55EFC
:102E750005855D5C8003122D82855C547553008049
:102E850041E55C9001BF12486FE0F55DE55C90019E
:102E9500DF12486FE0F55E900087E0F4042537F512
:102EA5005F900098E0FE900087E0F4042EF560E561
:102EB5005DB55E05855D5C8003122D82855C54756C
:102EC5005300022F719000BFE0D395375011E55C98
:102ED50090021F12486FE0F554755300022F719050
:102EE5000088E0D395375043E55C9001FF12486FA9
:102EF500E0F55DE55C90021F12486FE0F55E90001D
:102F050088E0F4042537F55F9000BFE0FE90008867
:102F1500E0F4042EF560E55DB55E05855D5C800336
:102F2500122D82855C547553008041E55C9001DF6C
:102F350012486FE0F55DE55C9001FF12486FE0F522
:102F45005E900098E0F4042537F55F900088E0FE78
:102F5500900098E0F4042EF560E55DB55E05855DAD
:102F65005C8003122D82855C54755300229000D03D
:102F7500E0F561756411753202753300AE24AF2535
:102F8500E56175F00FA4FDACF0EDD39FEC9E4021FB
:102F9500E5618E048F05FF120085ED75F010A4FF25
:102FA500AEF0E53775F01184FD7C00ED2FF56280FC
:102FB5000EE53775F01184FF7E00EF24F0F562858C
:102FC500625CE53775F01184AFF07E008F5F122DDE
:102FD50008855C63AE24AF259000D0E075F00FA4A2
:102FE500FDACF0EDD39FEC9E402875320275331091
:102FF50085625C122D0885635D855C5EAE24AF2518
:10300500E5618E048F05FF12484E8D5F8561601264
:103015002D82855C5275510075546475530022905C
:1030250000D0E0F561756411753202753300AE2488
:10303500AF25E56175F00FA4FDACF0EDD39FEC9ED7
:103045004021E5618E048F05FF120085ED75F010B6
:10305500A4FFAEF0E53975F01184FD7C00ED2FF588
:1030650062800EE53975F01184FF7E00EF24F0F5DE
:103075006285625CE53975F01184AFF07E008F5F83
:10308500122D08855C63AE24AF259000D0E075F065
:103095000FA4FDACF0EDD39FEC9E40287532027570
:1030A500331085625C122D0885635D855C5EAE24F8
:1030B500AF25E5618E048F05FF12484E8D5F856152
:1030C50060122D82855C5275510090009AE0B4041F
:1030D50053E53775F00484FF7E008F5CE53775F0A6
:1030E5000484ADF07C008D5F756404753201753321
:1030F50000E55CC3943F5005122D08800690019EA3
:10310500E0F55CAE51AF52E55C12483374648E0451
:103115008F05FF120085AE51AF52EF2DFDEE3CFC41
:103125008C518D5275546475530022900065E0B43E
:103135000146E53F75F00584FF7E008F5CE53F7530
:10314500F00584ADF07C008D5F75640575320575FD
:103155003300E55CC394175005122D0880069005D1
:1031650076E0F55CAE53AF54E55C2FFF50010E746D
:103175006412488A8E538F54900066E0B40146E588
:103185004075F00584FF7E008F5CE54075F0058491
:10319500ADF07C008D5F756405753205753348E5C6
:1031A5005CC394175005122D0880069005BEE0F506
:1031B5005CAE53AF54E55C2FFF50010E74641248AA
:1031C5008A8E538F54900075E0B40249E542C3944A
:1031D5004175F00584FF7E008F5CE54275F005843E
:1031E500ADF07C008D5F756405753206753300E5BD
:1031F5005CC394135005122D088006900672E0F505
:103205005CAE53AF54E55C2FFF50010E7464124859
:103215008A8E538F549000B7E0B4020280030232C5
:10322500CFE53775F01584FF7E008F5CE53775F0C7
:103235001584ADF07C008D5F7564157532037533AB
:10324500F4E55CC3940B5005122D08800690045ECE
:10325500E0F55CE55C75F0FFA4FFAEF09000B8E02A
:103265008E048F05FF120085ED90005AF0E53E753E
:10327500F078A4FFAEF074FF8E048F05FF12008571
:103285008C328D3374028C068D071248258F5CAC09
:1032950032AD337404FF12484E8D5F756404753288
:1032A5000675336EE55CC3941D5005122D08800626
:1032B5009006EAE0F55CAE53AF54E55C2FFF500194
:1032C5000E746412488A8E538F542290006DE0B4B8
:1032D50001179007A4E02554FFAE5350010E90004E
:1032E500C1E012488A8E538F5490006DE0B40316E6
:1032F500A201B3B35010900059E0C39405A824B8B7
:10330500000695254002801090008FE02554FFAE01
:103315005350010E8E538F54900067E0B402028023
:10332500030234FD90006AE0602FE53FD3941E4010
:1033350028900014E0FEA3E0FF9000A5E075F003DF
:10334500A4FDACF0EFD39DEE9C400E9000C9E0A823
:1033550024B80005D3952550030234FD9000B2E052
:103365008537F0A4FFAEF074051248337407124890
:10337500258E328F33900071E0A824B8000495257E
:103385005012900072E075F002A4FDACF0EFC39D01
:10339500EE9C40030234FDE53775F00B84FF7E009B
:1033A5009005EF12485AFEE0FFEE900069E0FEEF4F
:1033B5008E0088F0A4FFAEF074648E048F05FF12B2
:1033C50000858C328D33900031E075F018A4FFAE86
:1033D500F09000B0E08E048F05FF1200858C068DFD
:1033E5000790060712485AAE32AF33E012483374DD
:1033F500648E048F05FF1200858C328D33E53DA860
:1034050032B80077D395334072E53DC39533FFE479
:103415009532FE8E328F337428BE00039F500C7593
:103425003328753200740D900034F0AE32AF33900E
:10343500006AE012483374288E048F05FF12008558
:103445008C328D33AE51AF52740A8E048F05FF1244
:1034550000858D068C07AC32AD33CFCECF1200037D
:10346500740A8E048F05FF1200858C328D33AE51A0
:10347500AF521248928E518F52807DE53DA832B8E9
:10348500000495335072AE32AF33E53D12488A8E53
:10349500328F337428BE00039F500C753328753264
:1034A50000740D900034F0AE32AF3390006AE01234
:1034B500483374288E048F05FF1200858C328D33B6
:1034C500AE51AF52740A8E048F05FF1200858D062A
:1034D5008C07AC32AD33CFCECF120003740A8E0405
:1034E5008F05FF1200858C328D33AE51AF52EF2D13
:1034F500FDEE3CFC8C518D5222AE51AF52AC53AD1A
:103505005412000374648E048F05FF1200858C51DC
:103515008D52900062E08C068D0712483374648EDC
:10352500048F05FF1200858C518D52A2084017AEFD
:1035350024AF257405BE00039F5002D208E539D398
:1035450094CC4002D2029000C4E0B402089000C6B8
:10355500E0640160028017AE51AF52E54312483373
:1035650074E78E048F05FF1200858C518D529000F3
:1035750084E05402601B90007BE0A824B80012D3BD
:103585009525400DA208B3B35007E539C3949A4079
:10359500028028AE5AAF5B900079E075F002A4FD79
:1035A500ACF0EF2DFDEE3CFC74022DFD50010CE559
:1035B50039BC0007D39D400375680185395B755A91
:1035C50000E56870030236549000D7E0C395684063
:1035D50070E53F75F00584FF7E0090055F12485A3F
:1035E500E0F533753200AE32AF33900089E0124812
:1035F5003374648E048F05FF1200858C348D3590ED
:1036050000D7E004C395688C068D071248339000F7
:10361500D7E08E048F05FF1200858C348D35900020
:103625007AE08C068D07124833740A8E048F05FFE5
:10363500120085AE51AF52EF2DFDEE3CFC8C518D45
:103645005205689000D7E0C39568500375680090EF
:103655000084E05401601B900078E0A824B80012B3
:10366500D39525400DA208B3B35007E537C394CCD5
:1036750040028025900076E075F003A4FFAEF0E5EA
:10368500652FFF50010E74032FFF50010EE537BE65
:103695000007D39F4003756901853765E5697003A8
:1036A50002372F9000D8E0C395694070E53F75F06B
:1036B5000584FF7E0090055F12485AE0F5337532A8
:1036C50000AE32AF33900089E012483374648E0443
:1036D5008F05FF1200858C348D359000D8E004C32A
:1036E50095698C068D071248339000D8E08E048FBB
:1036F50005FF1200858C348D35900077E08C068DA2
:1037050007124833740A8E048F05FF120085AE51E7
:10371500AF52EF2DFDEE3CFC8C518D5205699000AA
:10372500D8E0C395695003756900900089E0A851F8
:10373500B8000495525009900089E0F55275510082
:10374500229000C5E0B401028003023851A208B3FB
:10375500500302384F900090E0B40168AE51AF526B
:10376500AC24AD25120003743C8E048F05FF1200B6
:10377500859000A0E0BC00109D400D9000A2E0A83F
:1037850051B8000495525002D203AE51AF52AC2449
:10379500AD25120003743C8E048F05FF1200859041
:1037A50000A0E0C3940ABC0015D39D40119000A26F
:1037B500E0C39405A851B80005D395525002800284
:1037C500C2038068AE51AF52AC24AD25120003741C
:1037D500788E048F05FF1200859000A0E0BC0010D4
:1037E5009D400D9000A2E0A851B8000495525004E8
:1037F500D2038038AE51AF52AC24AD25120003740C
:10380500788E048F05FF1200859000A0E0C3940A0E
:10381500BC0015D39D40119000A2E0C39405A851AA
:10382500B80005D3955250028002C203A203B340EB
:1038350019AE51AF529000A1E012483374648E0462
:103845008F05FF1200858C518D528002C2039000B6
:10385500C5E0B40258E53775F00884FF7E008F5C3B
:10386500E53775F00884ADF07C008D5F75640875EB
:1038750032017533E0E55CC3943F5005122D088095
:103885000690025EE0F55CE55C75F05EA4FFAEF0C7
:10389500740A8E048F05FF1200858C558D567402AF
:1038A500BC000AD39D4006755602755500A200B3AB
:1038B5004006A202B3B3500990001AE4F0A3F080C9
:1038C50024AE51AF527400D39F74019E400C9000FA
:1038D5001AE551F0A3E552F0800B74FF90001AF839
:1038E500E4F0E8A3F09000A7E0D394024006A20814
:1038F500B3B34002800DAE51AF5274021248338EFD
:10390500518F52900090E0B4010DAE51AF52740248
:103915001248338E518F52AE51AF52745E124833F6
:10392500740A8E048F05FF1200858C518D52740226
:10393500BC000AD39D4006755202755100900018CF
:10394500E551F0A3E552F022900031E090035F12BB
:10395500486FE0F566756764900031E0FE90009B66
:10396500E0D39E4037E53775F00884FF7E008F5C15
:10397500E53775F00884ADF07C008D5F75640875DA
:103985003203753396E55CC3941F5005122D0880EC
:1039950006900414E0F55C855C678035E53775F0C5
:1039A5000884FF7E008F5CE53775F00884ADF07CF8
:1039B500008D5F7564087532037533B6E55CC39495
:1039C5001F5005122D088006900434E0F55C855CD7
:1039D50067229000D1E0F561756411753204753385
:1039E50000AE24AF25E56175F00FA4FDACF0EDD375
:1039F5009FEC9E4021E5618E048F05FF120085ED49
:103A050075F010A4FFAEF0E53775F01184FD7C006C
:103A1500ED2FF562800EE53775F01184FF7E00EF1E
:103A250024F0F56285625CE53775F01184AFF07EB0
:103A3500008F5F122D08855C63AE24AF259000D101
:103A4500E075F00FA4FDACF0EDD39FEC9E4028751A
:103A5500320475331085625C122D0885635D855CC3
:103A65005EAE24AF25E5618E048F05FF12484E8DAD
:103A75005F856160122D82855C66756764229000A2
:103A8500D1E0F561756411753204753300AE24AF6C
:103A950025E56175F00FA4FDACF0EDD39FEC9E40DC
:103AA50021E5618E048F05FF120085ED75F010A4E8
:103AB500FFAEF0E53975F01184FD7C00ED2FF56260
:103AC500800EE53975F01184FF7E00EF24F0F56274
:103AD50085625CE53975F01184AFF07E008F5F1269
:103AE5002D08855C63AE24AF259000D1E075F00FFD
:103AF500A4FDACF0EDD39FEC9E40287532047533E0
:103B05001085625C122D0885635D855C5EAE24AF11
:103B150025E5618E048F05FF12484E8D5F85616036
:103B2500122D82855C667567649000CCE0B40479DB
:103B3500900031E0FE90009BE0D39E4037E537755D
:103B4500F00884FF7E008F5CE53775F00884ADF0E2
:103B55007C008D5F756408753203753396E55CC32B
:103B6500941F5005122D088006900414E0F55C851D
:103B75005C678035E53775F00884FF7E008F5CE56E
:103B85003775F00884ADF07C008D5F75640875327B
:103B9500037533B6E55CC3941F5005122D088006E6
:103BA500900434E0F55C855C6722900065E0B40123
:103BB5003BE53F75F00584FF7E008F5CE53F75F0C2
:103BC5000584ADF07C008D5F756405753205753330
:103BD50018E55CC394175005122D08800690058ED4
:103BE500E0F55CE567255CC39464F567900066E0E5
:103BF500B4013BE54075F00584FF7E008F5CE54030
:103C050075F00584ADF07C008D5F75640575320532
:103C1500753360E55CC394175005122D0880069036
:103C250005D6E0F55CE567255CC39464F567E56654
:103C35002567F55990006DE0B402109007A3E025C3
:103C450059FE9000C1E0F4042EF5599000C4E0D36C
:103C550094014040E543C394E7501D74E7C3954381
:103C6500FE9007A5E08E00F5F0E884FF7E008F5CEE
:103C7500E559255CF559801CE543C394E7FE90079B
:103C8500A5E08E00F5F0E884FF7E008F5CE559C362
:103C9500955CF559A2084006E5662464F559E55991
:103CA500D394644009E559C39464F5598003755963
:103CB5000090009DE0C39559500690009DE0F55990
:103CC50022D2009000B3E0A824B800049525503B0B
:103CD5009000B3E0A824B800049525500375590F4A
:103CE5009000B3E004A824B8000495255003755945
:103CF5000A9000B3E02402A824B8000495255005D5
:103D0500755905C2007409900034F07E017F00905A
:103D150000A3E01248339000B2E08E048F05FF1235
:103D25000085E537BC000CD39D4008C200740A909D
:103D35000034F09000A4E0C3953F500D9000B6E02C
:103D4500A824B80006952540028008C200740B908F
:103D55000034F0A200400375590590006DE0B403EE
:103D650006A201B3B34002802B900059E0C394052D
:103D7500A824B800049525500C90008EE0F55974E0
:103D85000C900034F0900059E0A824B80004952563
:103D95005002C20085594490005FE02559FE90000D
:103DA50031E075F01E84FC7F00EE2CF55922900061
:103DB50031E075F00584FF7E008F5C900031E07581
:103DC500F00584ADF07C008D5F7564057532037573
:103DD50033D69000B0E01475F00584FF7E00E55CF5
:103DE500BE00039F5005122D08800BE55C9004353D
:103DF50012486FE0F55CE55C9007A6F09007A6E039
:103E0500FE90009FE0C39E500890009FE09007A69B
:103E1500F022E53F75F00584FF7E0090055F1248AE
:103E25005AE0F56BE56BD394644010E56BC394647D
:103E350075F00F84FF7E008F6B8003756B0090001B
:103E450082E0256BF56B22900799E0FEA3E0FF74F5
:103E550004124825E537124833740F8E048F05FF89
:103E6500120085900797ECF0A3EDF0900075E0B493
:103E75000262E542C3944175F00584FF7E008F5CC4
:103E8500E54275F00584ADF07C008D5F75640575C0
:103E95003206753314E55CC394175005122D08805E
:103EA50006900686E0F55C900797E0FEA3E0FF74B8
:103EB5000A8E048F05FF120085E55C8C068D0712BE
:103EC5004833740A8E048F05FF120085900797EC1E
:103ED500F0A3EDF0900797E0FEA3E0FF90079DE0CB
:103EE500FCA3E0FDEDD39FEC9E400F90079DE0F80D
:103EF500A3E0900797C8F0A3C8F02290007CE0B437
:103F0500010385254F90007CE0B402129000B2E0D9
:103F15008537F0A4FFAEF074081248258F4F900046
:103F25007CE0B4030385394F90007CE0B40403853D
:103F35003F4F90007CE0B40507E540C39414F54F6E
:103F450090007CE0B4060385414F90007CE0B40707
:103F55000385424F90007CE0B4080385434F9000F1
:103F65007CE0B40903853E4F90007DE0FE90007E25
:103F7500E0D39E404B90007CE0B4041890007EE0B6
:103F8500C3954F5002D20490007DE0D3954F400277
:103F9500C204802A90007DE0C3954F500990007EB1
:103FA500E0D3954F50028002D20490007DE0D39576
:103FB5004F500990007EE0C3954F5002C204802AFD
:103FC50090007DE0D3954F400990007EE0C3954F6A
:103FD50040028002C20490007DE0C3954F400990E5
:103FE500007EE0D3954F4002D2042290007FE0B4DA
:103FF500010385254F90007FE0B402129000B2E0E6
:104005008537F0A4FFAEF074081248258F4F900055
:104015007FE0B4030385394F90007FE0B404038546
:104025003F4F90007FE0B40507E540C39414F54F7A
:1040350090007FE0B4060385414F90007FE0B40710
:104045000385424F90007FE0B4080385434F9000FD
:104055007FE0B40903853E4F900080E0FE9000812B
:10406500E0D39E4040900080E0C3954F50099000FA
:1040750081E0D3954F50028002D206900080E0D3B4
:10408500954F5009900081E0C3954F5002C20690AC
:10409500007FE0B401099000BEE0D395395002805D
:1040A50002C206802A900080E0D3954F4009900017
:1040B50081E0C3954F40028002C206900080E0C3B4
:1040C500954F4009900081E0D3954F4002D20622DA
:1040D500AE57AF5874F5D39F74019E4008785712B8
:1040E500489A0241D0755801755700AE24AF25E5B1
:1040F5006BBE000DD39F4009900094E0D3956C40B2
:1041050002801B756C00E56BC39525F54F900097F4
:10411500E0D3956A4006E56A254FF56A8002056C8D
:10412500900070E0D39539401CE537C395384015AC
:10413500AE24AF25E56BBE00039F5009900095E0C6
:10414500D3956D400280579007A7E0A824B80004D6
:1041550095255003756F009007A7E0A824B8000BBC
:10416500D395254006E5259007A7F0E56F702AE56C
:1041750025C3956BF54FE54FD394054003754F0562
:10418500900096E0C3956A5007E54FC3956A4002D3
:104195008007E56AC3954FF56A756D008002056D68
:1041A500E56F7016900070E0C39539500DE56B24EE
:1041B50005A824B8000695254002800F900083E0ED
:1041C500F56A756F0174789007A7F022AE57AF585E
:1041D50074E9D39F74039E4008785712489A0243A6
:1041E5007E755801755700756A32A21E402A756A98
:1041F50019900083E075F002A4FFAEF0E56CBE00F7
:1042050006D39F4002D21E056C756F037478900724
:10421500A7F0756E0002436DAE24AF25E56B6F4EBA
:10422500700302436DE56BBE000DD39F40099000FE
:1042350094E0D3956C40028017756C00A208B3B367
:104245005007E56FC3940340028003756A19800D1A
:10425500E56BC39525F54FE56C254FF56C90007022
:10426500E0D39539400E9007A7E0A824B80007D3FE
:1042750095254002800C056E900083E0B56E0375B0
:104285006F00E56FB4030DE56B2402A824B80006A2
:1042950095254002800A056EE56EB43C03756F02F4
:1042A500E56FB402299007A7E0A824B8000ED395BE
:1042B500254009E5259007A7F0756E00900070E090
:1042C500C395395009756E0074789007A7F0E56FAE
:1042D500705A900070E0D39539401CE537D3953876
:1042E5004015AE24AF25E56BBE00039F5009900035
:1042F50095E0D3956D40028008756D00756A4B8019
:1043050028E525C3956BF54FE54FD3940540037517
:104315004F05900070E0D395394008E56D254FF5C0
:104325006D8006E56D2406F56D756E00E56F7016FA
:10433500900070E0C39539500DE56B2405A824B8AD
:104345000006952540028003756F01E56FB40118DD
:10435500756A19056E900083E0B56E06756F027576
:104365006E0074789007A7F0E56A75F00AA4FFAEB1
:0A437500F09007A1EEF0A3EFF02294
:09486F002582F582500205832226
:0F48160025E050020583258250020583F582229A
:10006400EF2F500205832582F582E5833E2EF5832A
:010074002269
:10488A00CFC39FFF50011E22C3EF9DFFEE9CFE2265
:09487800E493F608740193F622A2
:08489A000806B6000218062210
:0D484100A3E004F07006124865E004F022C8
:0E003900A3E014F0B4FF06124865E014F022B4
:0E482500048007C3CE13CECF13CFD5E0F6220A
:10473500BC000FBE0008ED8FF084FFADF022E4FE53
:10474500FF22BE000DEF60FE54F0606F20E703020C
:1047550047EBEAC0E0EBC0E078017A0075F001EEC6
:1047650020E710EF25E0FFEE33FE0AC5F023C5F084
:1047750030E7F0EA5407F9096A7A007B006001081E
:10478500C3EC9E40167004ED9F4010ED9FFDEC9E1E
:10479500FCE5F0CA4ACA03F5F08005E5F003F5F03B
:1047A500C3EE13FEEF13FFD9D77908CACBCAD8D009
:1047B500EAFEEBFFD0E0FBD0E0FA22EC8FF084FCC0
:1047C500ED54F045F0C48FF084FEEDC454F045F08F
:1047D500C48FF084FDEEC4FE54F02DFFEE540F3C63
:1047E500FEADF07C0022790078008FF0EC7E082089
:1047F500E70DC3CD33CD33C933C9C833C8DEF08423
:1048050049F9E5F08FF0BE00E6FD7C00E9FFE8FE22
:014815002280
:0E483300F88FF0A4FFE5F0CE88F0A42EFE2250
:10000300EF8DF0A4F9A8F0EF8CF0A428F8EE8DF0B2
:06001300A428FEE9FF2213
:10007500600D782B02007F007830D8FED5E0F8229D
:10008500EEC0E07E00124735EFFDEEFCD0E0FE222B
:0C484E00EEC0E07E00124735D0E0FE22F4
:03001B0002001EC2
:03009B0002004917
:0300000002488132
:0948810075817075D000020393EB
:10485A00E5822FF582E5833EF583220582D5820221
:05486A001583158222F8
:10001E00C0E0C0F0C083C082C0D075D00012033ED5
:0B002E00D0D0D082D083D0F0D0E032E0
:10004900C0E0C0F0C083C082C0D075D000120341A7
:0B005900D0D0D082D083D0F0D0E032B5
:00000001FF
